:020000040000FA
:020000001029C5
:08000800FC00030EFD000408DA
:10001000FE000A08FF0000308A0083018B181528B3
:100020000B191D280C1828282F288B10201402309B
:10003000A0072E08031DAE032F280B1106308100E8
:10004000DA0B2F284030DB06DB176430DA002F286C
:100050000C1045088F0046088E00803086067F0809
:100060008A007E0884007D0E8300FC0E7C0E090051
:1000700039283A283B2808000617061638200612A9
:100080003820061308000612061738200616080046
:10009000EB000830EC000612EB1B061638200617A2
:1000A00038200613EB0DEC0B4B2883160616831233
:1000B0003820061738200000061383160612831214
:1000C00008000830EC008316061683123820061745
:1000D0000310061A0314EB0D38200613EC0B6628E8
:1000E0008316061283126B080800061206173820C2
:1000F0000613061608000616061738200613080011
:100100003C20D0304820A03004024820000848207D
:10011000840AE80B8628432008003C20D030482081
:10012000A030040248203C20D13048209828752077
:1001300061208000840AE80B97287B204320080078
:100140000030E900B830EA001230E8003C20D0303E
:100150004820B4208A110A124820EA0A0319E90A41
:10016000E80BA9284320080069088A006A08820071
:1001700000340034003400340634013401342134B6
:1001800000340034003400340034003400340034CF
:100190000034003483168612831286125327831686
:1001A00086168312F720E71BF62863308400B90116
:1001B0000530BC00BA010830BD00F720E71BF62867
:1001C0000521E71BF6280310BA0D04306702031857
:1001D0003A14BD0BDD283A08BC0BEF28F328800049
:1001E000840AB907DA283902031D671708000521B8
:1001F000E71B0429E7013427E70A861A04290A3095
:100200006702031CFB28E7170800E7013427E70A09
:10021000861E0F290A306702031C0629E71708000B
:1002200083018B012030A10003179E019F0103135E
:1002300083163F3085002030860008308700373035
:10024000950071308F00433081000C108312013013
:100250009000C0308B00061606170F30E000E20059
:100260006423F2308700A3210F2786130A30CA00C7
:100270000530CB00BE2194270A30CA000030CB00E5
:10028000D900BE21DD21D8010A30CF00B33084006F
:100290004F039D27B33084000830D3005308CA00B1
:1002A0000008CB00BE21840AD30B4E296227CF0B56
:1002B0004629DD21AE01DB01CD30A9000130AA00C5
:1002C0001430AB00DD30D60099276627F030870464
:1002D000DD21AF3084000130E8008D2083162F0827
:1002E0008312BB00BB1F87290230D8003430A9001D
:1002F0005630AA007830AB00FC30D600992726276C
:1003000033300505333A03198029A0206929D80123
:10031000AD01AC01DF01DC018030B100831720307A
:1003200084003C30BC008001840ABC0B93298313F9
:10033000A03084000730E8008D207323D0308B007C
:10034000A001AD17E8290F30CA000030CB00BE2154
:100350000930CA000030CB00BE210A30CA0000308C
:10036000CB00BE210B30CA000730CB00BE210C30C1
:10037000CA000130CB00BE21D6210800871006300C
:10038000CE004A08C9214B08C921CE0BC1298714C8
:100390000800CC000830CD000710CC1B071407154F
:1003A00000000711CC0DCD0BCC290800CB01083083
:1003B000CA00BE21CA0BD92908000C30CA00CB01E3
:1003C000BE2164270C30CA000130CB00BE210800DA
:1003D000AD1BEF292E08031D212A201C212AA03045
:1003E00084000730E8008D2073238A1575208A1158
:1003F000A01D0C2ACA20C03067050319052A8027D2
:10040000E701A011A01D022AFA295C0803190C2A91
:100410004F238A1575208A11AD132D08B8000319D2
:100420006C27B80303197027B80303197427B8039E
:1004300003197827B80303197C272010A011C926B7
:10044000DB26051CA523851CFB24851E0525871D91
:100450003D256B230F3062050F3A031D3122DB016E
:10046000E82925230319242B051A552A4B27051E95
:10047000372A6B230F3062050F3A031D392A5B19A7
:10048000DC0184270330D8005B080339A90045301C
:100490003B1C6730AA00F030D6009927D8013B18E2
:1004A00004273B1C1F276627222B621CA72A4B27E9
:1004B000DD016B230F3062050F3A031D592ADB174C
:1004C0003323DB1F7A2A8C27DD1E6A2A02305B1950
:1004D0000130772A5E08B900B90CB90E033039052E
:1004E000AB00390C7039AB04FE305B19FD30D6001F
:1004F0009927DB13051E8F2A6B230F3062050F3AF5
:100500000319602A4B275B08B90025230319222B06
:1005100039085B06031DDD01DD1ADD01592A4B2771
:10052000051E902A0330D8006730DD1A9C2A8827E0
:10053000DD035B19DC034530AA003030D600992773
:10054000D801DD1E0427DD1A1F276627592A6B23D1
:100550000F3062050F3A031DA72A4B270630810092
:100560006430DA000B118B16A901AA01AB01AF01AF
:10057000B0010A305B19AA00DB173323DB1FE52A21
:100580005B1BC62AFE305B19FD30E02AAF08031D55
:10059000CD2A3E305B193D30E02A01302F02031D89
:1005A000D52ACE305B19DD30E02A02302F02031D40
:1005B000DD2AF6305B19F530E02AFA305B19F930A4
:1005C000D6008A15FF218A11DB13051C0424851C23
:1005D0003324051E9E24851EEA2403303005031DA6
:1005E000DB17031D5B13B00104302F020319FC2A33
:1005F0006B236218BD2A1C2BDE010310AB0CDE0C32
:100600002B0CDE0CDE0CDE0403305B05DE049027D1
:1006100003180E2B5B19DC0A0427B42A0230D80019
:100620003430A900EF30AA00F030D60099272627F1
:10063000D8016B236218192B8B120B114B276B23DC
:10064000621C1F2BDB01AD170800DB01DB0AE21C7B
:10065000312BDB0A621D312BDB0A5B15E21D312BCE
:10066000DB015B080800201C4E2BA0308400073003
:10067000E8008D2073238A1575208A1120105C08EC
:1006800003194D2BA01D4E2BCA20C0306705031D3A
:100690004D2B4F238A1575208A11A011080065087B
:1006A0007F39C3006608C4003E260F304005C300F2
:1006B000C30E0F304105C3040F304205C400C40E01
:1006C0000A30C404DF1408003C204030482062088F
:1006D0004820432008003C20413048206120E200AF
:1006E0007B2043200800A03084000008A700840A73
:1006F0000008A600840A0008A500840A0008A800D3
:10070000840A0008A400840A00081F39A300840A90
:100710000008A200270803195F140800A030840015
:1007200027088000840A26088000840A25088000A3
:10073000840A28088000840A24088000840A230888
:100740008000840A2208800008004B270518012C2D
:100750003C30B8004D277F302D05031DB92B201CE0
:10076000B92BA03084000730E8008D2073236C275C
:1007700020100518BE2BB80BAA2BC72BAD0A0530CD
:100780002D020319AD01AD170230AE00012C0B1282
:100790000230D8002230A9000130AA002230AB007C
:1007A000FC30D6009927D801051CD42B0530AD00AC
:1007B000AF01B001A001301003302F020318E22B6B
:1007C0007027E32B6C27051C0424851C0D24051EB3
:1007D0007824851EEA2406302F020319F42B0330F7
:1007E00030050319E32BDB2B051CF42BB01CFE2B6F
:1007F0008E23A03084000730E8008020B001AD01D6
:100800000B16051C012C08004B270518092C301469
:10081000AF0A051C092C4B2708004B278518312CE3
:10082000B0142F08031D162C9F25212C01302F02F8
:10083000031D1C2C9525212C02302F02031D242C76
:100840004A255A26A800312C03302F02031D2A2CDA
:10085000E925312C04302F02031D302CD925312CF1
:10086000D125512708004B278518642CB0142F0878
:10087000031D3F2C5B1DF1255B196624642C0130A0
:100880002F02031D482C5B1DE1255B196F24642C8E
:1008900002302F02031D552C1030AB0780302B0285
:1008A000031C642C0F30AB05642CAB0A2B080F39EA
:1008B000B90002303902031C642C5B19622CAB0AAC
:1008C0002B1D642CF030AB05512708002930840023
:1008D0002B26A0302902031D6E2CA9010800103020
:1008E000AA07A0302A02031C772C0F30AA050800A3
:1008F0004B27051A9C2CB0142F08031D812CC225F0
:100900008C2C01302F02031D872CB6258C2C023035
:100910002F02031D8F2CA8255A26A8009C2C0330DB
:100920002F02031D952C17269C2C04302F02031D2B
:100930009B2C03269C2CF925512708004B27051AD0
:10094000CD2CB0142F08031DAA2C5B1D21265B198A
:10095000CF24CD2C01302F02031DB32C5B1D0D269F
:100960005B19DE24CD2C02302F02031DBE2C10306B
:10097000AB020318CD2C8030AB07CD2C2B080F39E0
:100980000319C92CAB032B080F39023C0319AB0325
:10099000CD2C03305B190130AB0451270800A903AB
:1009A000290A031DD62C6630A902DD2C29080F392F
:1009B0000F3C031DDD2C0630A9020800F0302A058B
:1009C0000319E52C1030AA02E92C0F30AA0590304B
:1009D000AA0408004B27851AF72C3014AF032F0AFE
:1009E000031DF72C0530DB08031D0330AF00851E07
:1009F000F72C4B2708004B278518012D0230AC0639
:100A0000AD17851C012D4B2708004B27851A2E2D6D
:100A100005302602031C232D55302602031C322DDF
:100A20000B12E9252508031D242D4A250130240237
:100A3000031D202D952501302302031D202D9F2508
:100A40005A26A800242D0B12A601A7018E23A03040
:100A500084000730E80080200B16AD17851E2E2D70
:100A60004B2708001430B8004D27851A2E2DB80BDF
:100A7000342D8A159E248A112E2D4B278719462D39
:100A80008030B106B11B0227B11F1F27871D462DDD
:100A90004B27080055252402031D512D0130A400C9
:100AA000542D243084002B26080002302302031D1D
:100AB000642D2208B4002108B3007825321C622D71
:100AC0002930772D2830772D043023020319762D15
:100AD000063023020319762D093023020319762DDF
:100AE000113023020319762D3130772D3030080074
:100AF000B201340888250339031D872D3408031DEE
:100B0000862D330888250339031D872D32140800EC
:100B1000BA003A0E0F39B9000310B90DB90DB90773
:100B2000B90D3A080F3939070800233084002B2605
:100B300013302302031D9E2D0130A3000800223034
:100B400084002B26A0302202031DA72DA20108003D
:100B5000A403031DAE2D5525A400B52D24080F397F
:100B60000F3C031DB52D0630A4020800A303031D8E
:100B7000BB2D1230C02D0F302302031DC12D0930B3
:100B8000A3000800A203220A031DC92D6630A20299
:100B9000D02D22080F390F3C031DD02D0630A202A4
:100BA0000800273084002B26603027020318A70195
:100BB0000800263084002B26603026020318A60188
:100BC00008002A3084002B2660302A020318AA016C
:100BD0000800253084002B26243025020318A501A7
:100BE0000800293084002B26243029020318A9018B
:100BF0000800273084003426F9302702031D022E16
:100C00005930A7000800263084003426F930260227
:100C1000031D0C2E5930A60008002A30840034260B
:100C2000F9302A02031D162E5930AA00080025307B
:100C300084003426F9302502031D202E2330A50020
:100C40000800293084003426F9302902031D2A2E99
:100C50002330A9000800800A00080F390A3C031D50
:100C6000080006308007080000080F3903193A2EE3
:100C700080030800800306308002080042308400B0
:100C80004626462646264626462608001030BC0044
:100C9000B9010310C40DC30DB90DF6303907031C9B
:100CA000532EB900C40ABC0B492E390830388000D5
:100CB000840308000130B400B3010130B6002108FC
:100CC0008825B70004303702031C6E2E031D6B2EDF
:100CD000220803196E2E0430B702622E2208340255
:100CE000031D762E3708330203198B2E0130B60709
:100CF00078253218B60A073036020318B6003430A9
:100D000084002B26A0303402031D6E2EB401333034
:100D100084002B266E2E0130B500230835020319FE
:100D2000A52E35088825BA00B226B607023035024E
:100D3000031D9D2E78253218B60A07303602031897
:100D4000B600353084002B268D2E24088825B60762
:100D5000B60307303602031CAF2EB600A92EB60A22
:100D6000360808003A03D5000630D400BE30D50757
:100D70000318D40A54088A0055088200033400344A
:100D800003340234033402340334033402340334AE
:100D90000234B11FDA2E59302602031DD52E5730EA
:100DA0002702031CD52E3115DA2E27082604031D31
:100DB000DA2EB11508007F3031050319F02E311CF1
:100DC000E32E0D27EE2EB11CE82E1F271F27EE2E37
:100DD000311DEC2EF126EE2EF82686138030B1055B
:100DE0000800F730C5001F30C60064302A2708000D
:100DF000FB26FB26FB26FB30C5009030C600FA30F0
:100E00002A27080006274B2706274B27F630C50060
:100E10000930C60064302A2708000F274B27062711
:100E20004B27F830C5008930C60064302A270800F7
:100E3000F130C5001230C60064302A270800F130B6
:100E4000C5001230C600FA302A27080018274F279D
:100E50001F27080083160C148312542783160C10C6
:100E60008312B11D861308000430C7000000C70BB1
:100E7000362F000008000F30C7003E2FC70B3D2F54
:100E8000412F08002730C700452FC70B442F482F9C
:100E900008000A30542F1E30542F3230542F643043
:100EA000542FC830542F0130C800DD30C700582FF0
:100EB000592F5A2FC70B572F00005E2F5F2FC80BDB
:100EC000552F08000530672F0A30672F1E30C900E4
:100ED0004F27C90B682F08008A151A218A110800AC
:100EE0008A1552218A1108008A1586218A11080064
:100EF0008A15A7218A1108008A15C8218A110800BD
:100F00008A15E8218A1108008A151C208A11080018
:100F10008A1531208A1108008A1537208A110800A5
:100F20008A155C208A1108008A15D92402258A11A5
:100F300008008A15FF218A1108008A1583228A1168
:020F40000800A7
:101000008A112B268A1508008A1134268A150800B1
:101010008A113E268A1508008A11C9218A150800FE
:101020008A1149278A1508008A114B278A1508005A
:101030008A1126278A150800BB01831720308400F7
:101040001430BC00801F2B285B0800060339031DE9
:101050002B2880013B1403308407BC0B2228831308
:1010600008008317610884008001831308005D086D
:10107000B9008317203084001430BC00801F492839
:101080005B0800060339031D4928390803194F2856
:10109000B90303308407BC0B3E28DD165A28040828
:1010A000E1000008DE00840A0008A900840A0008A4
:1010B000AA00DD0A8313080083172030840014304F
:1010C000BC00801F692803308407BC0B612803140F
:1010D0007328DE175E088000840A29088000840ACD
:1010E0002A08800003108313080003305F050319EA
:1010F00019292808B6000310B60DB60D8317203045
:1011000084001430BC00801F122900081C39031908
:101110008C283606031D12290008DE00840ADF1C15
:10112000A02803305E05033A031D1329000843027B
:10113000031D1329840A000844020319AA2814294C
:1011400000087F392502031D1329840A000826029E
:10115000031D14295E080339BD001030B900BD031A
:101160000319B5280310B90DAF286008BA00390873
:10117000DE1AE004FF3ADE1EE0056008E2008A1194
:1011800064238A15B11FCF285F18CB283A08600660
:10119000403903191429DE1A3114DE1EB114DF1888
:1011A00014298403801FDB285E1FD828DE1ADD285F
:1011B0008403800112295E1F1329840320308006D6
:1011C000840ADE1AF5280420F9300002031D1329D1
:1011D000233080001C30DE05031913290430DE02A1
:1011E000031D0D291C30DE000D290008B9008013F5
:1011F00000202430000203188001B91B80177F30C3
:101200000005031D13291C30DE05031913290430C2
:10121000DE07DE1E0D290430DE008403E330800586
:101220005E088004840A840A840ABC0B8328831322
:10123000DF0108002508A900AC1838212608AA00FB
:101240002708AB0005302D02FE30031D2F29043086
:101250002F02323003192F29C23003180E30D60066
:10126000AC1C3629F03029050319D613FF210800DC
:101270002C102908031D3F291230A90051291230D2
:101280002902031C51292C1403195129A9000E30DD
:101290002902031C51291030290203185129063054
:1012A000A9020800A01868292208A9002308AA009A
:1012B0002408AB0005302D02FD30031D7B290130D1
:1012C0002F02313003197B29C13003180D307B29DF
:1012D0000130D8000E30A9002803D5000930D40011
:1012E0007F30D5070318D40ABA22AA0009308A0031
:1012F000F030AB007830D600FF21D801080001346F
:101300002334453467348934AB34CD3465087F39B0
:10131000C3006608C4000820A9013D30D600E51FBF
:1013200094290E30A9005617AA0130304002031943
:101330009C29AA00AA0ED6160F304105AA040F3028
:101340004205AB00AB0E0A30AB04FF210800630876
:10135000C3006408C4000820A9011D30D600303045
:101360003F020319B529A9005617AA0130304002DF
:101370000319BD29AA00AA0ED6160F304105AA04EA
:101380000F304205AB00AB0E0B30AB04FF21080061
:1013900005302702031CE629153027020318D2293D
:1013A0005221E72925302702031CE6293530270280
:1013B0000318DC298621E72945302702031CE6298A
:1013C000553027020318E629A721E7291A2108002A
:1013D0000230D800E71FF3293430A9009A30AA0060
:1013E000BC30AB00F9293430A9009A30AA00BD30D6
:1013F000AB00FC30D600FF211820D8010800522A8B
:101400002E080319102AB33084000830CF002D0AAB
:101410004F0200300319FF308000840ACF0B072AE7
:10142000DB308400D7000830D30087100630CE00B0
:1014300053080C2000080C2008308402CE0B182A18
:101440008714D70A57088400D30B152A073087055D
:10145000D61C412AC030DB1B4F2AF030AC1C4F2A6F
:1014600005302D02031D392AB030AC1C4F2A7030D4
:101470004F2AF030A01C4F2A70302C1C4F2AB0305D
:101480004F2A0030561C4F2A05302D0203194E2AD0
:101490004030DB1B4F2A1030561F4F2A5030F03A95
:1014A00087040800B3308400D61F592A290E8322EE
:1014B0005A2A7B22561F5F2A29088322602A7B2210
:1014C000D61E652A2A0E8322662A7B22561E6B2A86
:1014D0002A0883226C2A7B22D61D712A2B0E832296
:1014E000722A7B22D91BD801561D792A2B08832208
:1014F0007A2A7B22002A0830BD0003018000840A7A
:10150000BD0B7D2A08000F39D5000310D50DD50D70
:10151000D50D5808031D902A0A30D400BE30A22AE7
:10152000B900B903031D982A0B30D4003630A22A23
:10153000B903031D9F2A0B30D400B630A22A0C3009
:10154000D4003630D5070318D40A0830BD00BA22BB
:10155000B9000A308A000830BC00B90DBA0CBC0BC7
:10156000AD2A3A088000840AD50A0319D40ABD0BB3
:10157000A72A080054088A00550882007C34C63423
:10158000C634C634C634C634C6347C341834383411
:10159000183418341834183418343C347C34C634B5
:1015A000C6340C34183430346034FE347C34C634E1
:1015B0000C3438340C34C634C6347C3418343834E3
:1015C0005834D834D834FE3418341834FC34C03489
:1015D000C034FC3406340634C6347C347C34C6341F
:1015E000C034FC34C634C634C6347C34FE34C6340D
:1015F00006340C3418343034303430347C34C6344F
:10160000C6347C34C634C634C6347C347C34C634E8
:10161000C634C6347E340634C6347C34CE34D13439
:10162000303430343034303431341E34E234A43485
:10163000E834103410342E344A348E34C634C63470
:10164000C634C634C6346C343834103400340034F4
:10165000003465349634F434843464340034003413
:1016600000340034FE340034003400340034643478
:1016700094348434643414341434E3340034A234A1
:10168000A234B234AA34A634A234223400348934C9
:10169000DA34AA34AA348A348A348934003491344E
:1016A0005134593455345334513491340034FA346C
:1016B00022342234223422342234213400345E3461
:1016C000503450345C34503450349E3400348B34B5
:1016D0008A348A34AB34AA34AA3453340034DC3428
:1016E00012341234923412341234DC340034FA34AA
:1016F000223422342334223422342234003452342B
:1017000052345234D234523452344C3400347B3458
:1017100042344234733442344234423400349C34D0
:10172000483448348834483448345C3400346334B2
:1017300094348434643417341434E43400343E3440
:1017400088348834883488348834883400340234C7
:101750000434083408340834043402340034803447
:101760004034203420342034403480340034673412
:1017700094348434673414341434E7340034BE347D
:101780000834083408340834083488340034003409
:101790001034543438345434103400340034F034B9
:1017A00080348534E63484348434F43400340034B2
:1017B0000034AC343034203420342134003401344B
:1017C0000134013401340134013401340034C634AD
:1017D00029342834263421342134CE34003466347C
:1017E000993411342234143498346F340034623410
:1017F0009634123422341234923467340034723402
:101800004A344A344B344A344A34723400345F34F4
:1018100044344434C43444344434443400346634AA
:1018200099341134223444348834FF340034E6349B
:101830004934493449344934493446340034CF3486
:10184000A834A834CE34883488348F3400348B34B0
:10185000DA34AA34AB348A348A348B340034D13449
:101860001B341534953411341134D13400343234EE
:101870004A344234433442344A34323400344434F7
:101880004C344434C434443444344E3400344C3442
:1018900052344234C434483450345E3400344C340E
:1018A00052344234C434423452344C34003432342E
:1018B0004A344234423442344A34333400341C34DF
:1018C000123412341C3412341234D23400348934B9
:1018D0008A34CA34AA349A348A34893400349F341E
:1018E0004434443444344434443484340034703410
:1018F00048344A3473344A344A3472340034083435
:101900000034D8340834083408341D3400348034AA
:1019100080348334843487348434F33400340034A2
:1019200000342234A234A234143408340034003495
:10193000003438340034383400340034D9170A30D5
:10194000CA0059080F39CB008A11BE218A1503300D
:10195000D8008930A900AB30AA00C030AB005908CC
:101960000F39AB04FC30D600FF21D913851CC024ED
:10197000051ECD24D91B9F2C851EB62CAD17080043
:1019800014208518C92CD90A0A3059020318D90322
:10199000D917851CC92C142008001420051AD52C31
:1019A000D903590A0319D901D917051ED52C1420BA
:1019B00008000230D0000301232503013B2501303C
:1019C0003B2501302F2501304825030148250230F1
:1019D000232502303B2503303B2503302F250330E0
:1019E0004825023048250430232504303B250530A6
:1019F0003B2505302F250530482504304825D00BE0
:101A0000DB2C08000330D0000301232503013B2514
:101A100001303B2502303B2503303B2504303B257C
:101A200005303B2505302F25053048250430482555
:101A30000330482502304825013048250301482558
:101A4000D00B042D0800D1000130D3000130D200AA
:101A50000830CF005525D30ACF0B2A2D0800D1001E
:101A60000830D3008030D2000830CF005525D30392
:101A7000CF0B362D0800D1000830D3000130D20042
:101A80000830CF0055250310D20DCF0B422D080092
:101A9000D1000130D3008030D2000830CF0055256E
:101AA0000310D20CCF0B4F2D080087105108053CB6
:101AB0006D2553080C2052080C2051086D25871401
:101AC000102087105108053C6D2553080C20030198
:101AD0000C2051086D2587140800CE004E0803190C
:101AE000772D03010C2003010C20CE0B712D080073
:02400E00C43CB0
:1042000043006F0070007900720069006700680069
:1042100074002000280043002900200032003000F4
:10422000320031002D003200300032003200200018
:104230006200790020004D002E00590061006D00E1
:0C42400061006D006F0074006F00FF0053
:00000001FF
